:1000000000308A0030280000930100347F309300D4
:1000100000342B308400000803191B280230A10093
:10002000A001A00B1128A10B10289730A000A00B55
:100030001728800B0E2800340C30A1001F08C3398C
:1000400021049F000D30A000A00B24289F149F18AE
:10005000272883161E088312A5001E08A6008228E2
:1000600084011F3083051F1383161F149F141F154F
:100070009F15073083129F00703083168F00183051
:10008000650070308F0007308312990083160508D1
:1000900006308312A000A00B4B28000019088C1119
:1000A0001F1383161F109F101F119F151F129F16DD
:1000B0001F1383129F171F14831605118312051136
:1000C0000C3095000030A10005389200FF308316F7
:1000D0009200C03083128B0485120420A9012908E4
:1000E000023C031C7F2885160620FA30AB0009204D
:1000F00085120420FA30AB000920A90A6F28851266
:1001000004201C282608033C031C9A28031D8C2865
:100110002508213C031C9A28851606200230AA00D7
:10012000FA30AB000920AA0B90288512FA30AB00F8
:100130000920FE282608033C031CB328031DA4281D
:1001400025083D3C031CB328851606200230AA0072
:10015000FA30AB000920AA0BA82885120420FA3037
:10016000AB000920FE282608033C031CCC28031DF5
:10017000BD282508663C031CCC2885160620FA30CD
:10018000AB000920851204200230AA00FA30AB002F
:100190000920AA0BC628FE282608033C031CE528D4
:1001A000031DD6282508823C031CE5288516062059
:1001B000FA30AB000920851204200430AA00FA307E
:1001C000AB000920AA0BDF28FE282608033C031CED
:1001D000FC28031DEF2825089E3C031CFC288516DF
:1001E000FA30AB00092085120230AA00FA30AB00C9
:1001F0000920AA0BF628FE28851204208128630016
:02400E00C43FAD
:00000001FF
